:100B92000000F88BF8F2F95BF9B7FA14FA66FAB9C1
:100BA200FB03FB4AFB8FFBCFFC0BFC43FC78FCAB4B
:100BB200FCDBFD08FD33FD5BFD81FDA5FDC7FDE707
:100BC200FE05FE21FE3CFE55FE6DFE84FE99FEAD45
:100BD200FEC0FE02FEE3FEF3FF02FF10FF1DFF2A2E
:100BE200FF36FF42FF4CFF56FF60FF69FF71FF793E
:100BF200FF81FFFF00040D080F0811080D080D0802
:100C02000F0811080D08110812081408000811082D
:100C1200120814080008140616021406120211081B
:100C22000D08140616021406120211080D080F0808
:100C320008080D0800080F0808080D080008FFFF43
:0A0C4200C0F9A4B0999282F88090E6
:1010DC00015001015101015200C10A0127020153C3
:1010EC0001015405014F3C0126FF0124FF012AFF99
:1010FC000129FF012B00014500014E0001250001D3
:10110C0028FFC10DC106C1030747000012160729AD
:07111C002401220101230060
:06120F00C290C292D290D1
:0F121500EF7F08A2E09291D292C292C313DFF44E
:0112240022A7
:0F1270007F08C313A29192E7D292C292DFF4FFDC
:01127F00224C
:04123900E4FD7F8EC3
:0F123D00AE0512120FAF06121215D292C29022F6
:0A000E0012120F121270D292C2906B
:0100180022C5
:101186007508801212397C07120972FDAF08121217
:101196003D740129F9E43AFA05080508DCEA7D8080
:0511A6007F8E02123DE6
:100FFA007F8112000EEF12098B7F8312000E900080
:10100A0001EF12099D7F8512000E900002EF12096E
:10101A009D7F8B12000E900003EF12099D7F8712AD
:10102A00000E900004EF12099D7F8912000E9000B5
:10103A0005EF12099D7F8D12000E900006EF02093E
:01104A009D08
:0211D0008F0A84
:1011D200E50AD394004017750BB51207F57F5BDF64
:0E11E200FE150BE50BD3940050F0150A80E2C9
:0111F00022DC
:10122500750A961207F57F50DFFE150AE50AD39475
:031235000050F076
:011238002293
:03000B00021124BB
:10112400C0E0C083C082C0D0B297E55025E02492CD
:10113400F582E4340BF583E493F58CE55025E02443
:1011440093F582E4340BF583E493F58AD0D0D0820E
:05115400D083D0E03261
:100CF500E4F508F509E5277003020D8BE550B4FF0F
:100D050005E551F46074E50825E024F6F582E43440
:100D15000BF583E493F550E50825E024F7F582E427
:100D2500340BF583E493F551E550B4FF07E551B471
:100D3500FF021527E5507004C28C8035E550B4FFDD
:100D45000CC28C7F1E1211D0E4F50880AFE5082592
:100D5500E024F8F582E4340BF583E493B55010D222
:100D65008CAF511211D0C28C1212250508808DD27C
:100D75008CAF511211D005088082E4F50875500139
:090D8500755101020CFA752702F8
:010D8E002242
:0D11F100EFC43333335480447FF5807F0A10
:1011FE00E4FEEEC39F5009E4FD0DBD32FC0E80F2FD
:01120E0022BD
:10001E00E508652C6005B20C852C08300623E52812
:10002E0070028017E528B401028005E528B40205A8
:10003E007552058008E528B40307E4F552D20BD2B9
:10004E0001E552147003020379147003020476144E
:10005E00700302068014700302017314700302050C
:10006E0073240560030207F4A20B82025028C2A774
:10007E003087047F0180027F001211F1D2A7C2A641
:10008E003087047F0180027F00EFC4333333548006
:10009E00447FF5808048E52EC4540F900C42935453
:1000AE007FFF3087047E0180027E00EEC43333333F
:1000BE0054804FF580C2A77F0A1211FED2A7E52EFB
:1000CE00540F900C4293547FFF3087047E018002C0
:1000DE007E00EEC433333354804FF580C2A67F0AC0
:1000EE001211FED2A6A20182025028C2A5308704A8
:1000FE007F0180027F001211F1D2A5C2A4308704C5
:10010E007F0180027F00EFC43333335480447FF588
:10011E00808048E52DC4540F900C4293547FFF30DD
:10012E0087047E0180027E00EEC433333354804F49
:10013E00F580C2A57F0A1211FED2A5E52D540F90AF
:10014E000C4293547FFF3087047E0180027E00EEC6
:10015E00C433333354804FF580C2A47F0A1211FE8C
:10016E00D2A4020677E546C39414400302027CA291
:10017E000B82025028C2A73087047F0180027F00C5
:10018E001211F1D2A7C2A63087047F0180027F0030
:10019E00EFC43333335480447FF5808048E52EC45A
:1001AE00540F900C4293547FFF3087047E018002DF
:1001BE007E00EEC433333354804FF580C2A77F0ADE
:1001CE001211FED2A7E52E540F900C4293547FFFCE
:1001DE003087047E0180027E00EEC43333335480B8
:1001EE004FF580C2A67F0A1211FED2A6A20182028C
:1001FE005028C2A53087047F0180027F001211F1C2
:10020E00D2A5C2A43087047F0180027F00EFC433E1
:10021E0033335480447FF580804AE52DC4540F90CB
:10022E000C4293547FFF3087047E0180027E00EEE5
:10023E00C433333354804FF580F580C2A57F0A1244
:10024E0011FED2A5E52D540F900C4293547FFF3032
:10025E0087047E0180027E00EEC433333354804F18
:10026E00F580C2A47F0A1211FED2A4020677A20460
:10027E0082025028C2A73087047F0180027F0012BD
:10028E0011F1D2A7C2A63087047F0180027F00EF52
:10029E00C43333335480447FF5808048E531C454F1
:1002AE000F900C4293547FFF3087047E0180027EB4
:1002BE0000EEC433333354804FF580C2A77F0A1249
:1002CE0011FED2A7E531540F900C4293547FFF30AC
:1002DE0087047E0180027E00EEC433333354804F98
:1002EE00F580C2A67F0A1211FED2A6A20782025084
:1002FE0028C2A53087047F0180027F001211F1D23F
:10030E00A5C2A43087047F0180027F00EFC433337F
:10031E00335480447FF5808048E530C4540F900CF0
:10032E004293547FFF3087047E0180027E00EEC42C
:10033E0033333354804FF580C2A57F0A1211FED29B
:10034E00A5E530540F900C4293547FFF3087047E06
:10035E000180027E00EEC433333354804FF580C2E9
:10036E00A47F0A1211FED2A40207EBA20182025050
:10037E0028C2A73087047F0180027F001211F1D2BC
:10038E00A7C2A63087047F0180027F00EFC43333FB
:10039E00335480447FF5808048E52DC4540F900C73
:1003AE004293547FFF3087047E0180027E00EEC4AC
:1003BE0033333354804FF580C2A77F0A1211FED219
:1003CE00A7E52D540F900C4293547FFF3087047E87
:1003DE000180027E00EEC433333354804FF580C269
:1003EE00A67F0A1211FED2A6A20082025028C2A532
:1003FE003087047F0180027F001211F1D2A5C2A4C2
:10040E003087047F0180027F00EFC4333333548082
:10041E00447FF5808048E52CC4540F900C429354D1
:10042E007FFF3087047E0180027E00EEC4333333BB
:10043E0054804FF580C2A57F0A1211FED2A5E52C7D
:10044E00540F900C4293547FFF3087047E0180023C
:10045E007E00EEC433333354804FF580C2A47F0A3E
:10046E001211FED2A4020677A20482025028C2A75D
:10047E003087047F0180027F001211F1D2A7C2A63D
:10048E003087047F0180027F00EFC4333333548002
:10049E00447FF5808048E531C4540F900C4293544C
:1004AE007FFF3087047E0180027E00EEC43333333B
:1004BE0054804FF580C2A77F0A1211FED2A7E531F4
:1004CE00540F900C4293547FFF3087047E018002BC
:1004DE007E00EEC433333354804FF580C2A67F0ABC
:1004EE001211FED2A6A20782025028C2A53087049E
:1004FE007F0180027F001211F1D2A5C2A4308704C1
:10050E007F0180027F00EFC43333335480447FF584
:10051E00808048E530C4540F900C4293547FFF30D6
:10052E0087047E0180027E00EEC433333354804F45
:10053E00F580C2A57F0A1211FED2A5E530540F90A8
:10054E000C4293547FFF3087047E0180027E00EEC2
:10055E00C433333354804FF580C2A47F0A1211FE88
:10056E00D2A40207EBA20B82025028C2A730870446
:10057E007F0180027F001211F1D2A7C2A63087043C
:10058E007F0180027F00EFC43333335480447FF504
:10059E0080804DE52A75F00A84900C4293547FFFBB
:1005AE003087047E0180027E00EEC43333335480E4
:1005BE004FF580C2A77F0A1211FED2A7E52A75F069
:1005CE000A84E5F0900C4293547FFF3087047E013D
:1005DE0080027E00EEC433333354804FF580C2A6C2
:1005EE007F0A1211FED2A6A20182025028C2A530A5
:1005FE0087047F0180027F001211F1D2A5C2A430C0
:10060E0087047F0180027F00EFC43333335480446C
:10061E007FF580804DE52975F00A84900C42935445
:10062E007FFF3087047E0180027E00EEC4333333B9
:10063E0054804FF580C2A57F0A1211FED2A5E5297E
:10064E0075F00A84E5F0900C4293547FFF308704D6
:10065E007E0180027E00EEC433333354804FF5802A
:10066E00C2A47F0A1211FED2A4A20C929392870208
:10067E0007EFE532C4540F75F00AA4FFE532540FAC
:10068E002FFBA20882025028C2A73087047F018068
:10069E00027F001211F1D2A7C2A63087047F01801B
:1006AE00027F00EFC43333335480447FF580807B68
:1006BE00EB24C6FFE43407FE7C037DE81209BF7C01
:1006CE00007D0A1209BF74422DF582740C3CF5832D
:1006DE00E493547FFF3087047E0180027E00EEC4D7
:1006EE0033333354804FF580C2A77F0A1211FED2E6
:1006FE00A7EB24C6FFE43407FE7C007D641209BF1D
:10070E007C007D0A1209BF74422DF582740C3CF5F3
:10071E0083E493547FFF3087047E0180027E00EED7
:10072E00C433333354804FF580C2A67F0A1211FEB4
:10073E00D2A6A20982025028C2A53087047F01806A
:10074E00027F001211F1D2A5C2A43087047F01806E
:10075E00027F00EFC43333335480447FF5808076BC
:10076E00EB24C6FFE43407FE7C007D0A1209BF7C31
:10077E00007D0A1209BF74422DF582740C3CF5837C
:10078E00E493547FFF3087047E0180027E00EEC426
:10079E0033333354804FF580C2A57F0A1211FED237
:1007AE00A5AF03EB24C6FFE43407FE7C007D0A12DE
:1007BE0009BF74422DF582740C3CF583E493547F8B
:1007CE00FF3087047E0180027E00EEC43333335443
:1007DE00804FF580C2A47F0A1211FED2A4D293D20A
:0607EE00877F0A1211FED4
:0107F40022E2
:1007F500E50C652C6005B20C852C0C30A00930A1E8
:100805000630A20320A3157550FF7551FFE4F527A7
:10081500C28CC297C20A755301755405E52224FEA0
:1008250060541470030208B51470030208F01470C4
:100835000302092A2404600302094FD2A430870465
:100845007F0180027F00EFC43333335480447FF54A
:1008550080E52EC4540F900C4293547FFF308704DB
:100865007E0180027E00EEC433333354804FF58021
:10087500C2A775220222D2A73087047F0180027F9A
:1008850000EFC43333335480447FF580E52E540F95
:10089500900C4293547FFF3087047E0180027E00D6
:1008A500EEC433333354804FF580C2A6752203223C
:1008B500D2A63087047F0180027F00EFC433333333
:1008C5005480447FF580E52DC4540F900C42935419
:1008D5007FFF3087047E0180027E00EEC433333310
:1008E50054804FF580C2A575220422D2A530870415
:1008F5007F0180027F00EFC43333335480447FF59A
:1009050080E52D540F900C4293547FFF3087047E71
:100915000180027E00EEC433333354804FF580C22C
:10092500A475220522A20C929392873087047F0139
:1009350080027F00EFC43333335480447FF580D287
:0A094500A4D2A5D2A6D2A775220104
:01094F002285
:10109400BF01067B17E4FC8007BF02047B3BE4FC32
:1010A400BF0104AE2A8005BF0202AE29ED70031E03
:1010B40080010ED3EB6480F8EE6480984002AE04A5
:1010C400C3EC6480F8EE6480985002AE03BF010262
:0710D4008E2ABF02028E29E3
:0110DB0022F2
:100F1B0012001E20A21420A20512001E80F87526B6
:100F2B00FF7524FFC20AD206C20320A13820A105F7
:100F3B0012001E80F8E52A75F00A84C454F0FFE510
:100F4B002A75F00A84EF25F0F526E52975F00A8459
:100F5B00C454F0FFE52975F00A84EF25F0F524D28F
:100F6B000AD206C20320A31920A30512001E80F883
:100F7B007526FF7524FFC20AC203E4F552C20BC2E9
:020F8B00012241
:10104B0012001E20A21120A20512001E80F8E4F54A
:10105B004EFDAF2B12109420A11220A10512001EE1
:10106B0080F8E4F54E7D01AF2B12109420A31920CC
:10107B00A30512001E80F87526FF7524FFC20AC255
:09108B0003E4F552C20BC201227C
:100F8D00D203D206752B017901E52EC4540F75F0ED
:100F9D000AA4FFE52E540F2FF52AE52DC4540F7525
:100FAD00F00AA4FFE52D540F2FF52930033E20A0A4
:100FBD001920A00512001E80F8E4F54E09E9D3941E
:100FCD00024002E4F9892B755205E52B7007C20B1F
:100FDD00C201120F1BE52BB40104D20B8009E52BC6
:0C0FED00B402C8C20BD20112104B80BF2E
:010FF90022D5
:100AD50012001E20A05720A00512001E80F8E4F584
:100AE5004E052BE52BD394074003E4F52BE52BB4FA
:100AF50008005039900B00F8282873020B18020BD8
:100B05001A020B1C020B21020B23020B28020B28D5
:100B1500020B2F80028000E4F5528011800075528F
:100B250002800A80007552038003755205E52BB4D7
:100B350008005058900B40F8282873020B58020BF8
:100B450069020B6D020B73020B79020B7F020B8599
:100B5500020B8CC20BC201C200C204C207C208C28A
:100B650009020EA3D20B801CC20BD2018016C20152
:100B7500D2048010C204D207800AC207D2088004BA
:0D0B8500C208D209021159C209120F8D22B7
:1011590012001E20A21120A20512001E80F8E4F53B
:101169004EFDAF2B120C4C20A11220A10512001E1E
:0D11790080F8E4F54E7D01AF2B120C4C22E6
:100EA30012001E20A23020A20512001E80F8052386
:100EB300D3E523648094824003E4F523E52370049F
:100EC300F5528012E523B401057552048008E52329
:100ED300B4020375520120A13020A10512001E8027
:100EE300F81523C3E523648094805003752302E53A
:100EF300237004F5528012E523B401057552048072
:100F030008E523B4020375520120A30B20A30512A5
:070F1300001E80F8120F8D93
:010F1A0022B4
:020C4C008D0811
:100C4E00EF24FE601814601D1460221460271460D7
:100C5E002C2405702E7C847917E4FB80267C827907
:100C6E003BE4FB801E7C88790C7B0180167C8679A8
:100C7E001FE4FB800E7C8C79147B1480067C8C79AF
:100C8E0063E4FBEC4401FF12000EEFC4540F75F049
:100C9E000AA4FEEC4401FF12000EEF540F2EFAE5EB
:100CAE000870031A80010AD3E96480F8EA64809818
:100CBE004002AA03C3EB6480F8EA6480985002AA4B
:100CCE0001121239AF04EA75F00A120950C454F039
:100CDE00FEEA75F00A120950ADF0EE2DFD12123D2E
:070CEE007D807F8E02123DA4
:1011AB00AC05AB07121239AF03EC75F00A84C454CB
:1011BB00F0FEEC75F00A84E5F04EFD12123D7D80D9
:0511CB007F8E02123DC1
:10124C007F8112000EEF30E708543FFD7F801211B2
:01125C00ABE6
:01125D00226E
:03001B00020E1BB7
:100E1B00C0E0C0D075D000758D3C758BAF05450516
:100E2B004E0525300629E528D394035022AF4F15E4
:100E3B004FEF701B754F3CC2067528FF30030975C9
:100E4B005205D20BC2018007755200C20BC201E5DD
:100E5B0045C394094014B202E528D39403400375AB
:100E6B0028003006020528754500E525C39413407C
:100E7B0011752500B2050546E546D3941940037557
:100E8B004600E54ED394C8400A754E00E52B60032F
:080E9B00752B00D0D0D0E0322D
:10125E00758911758D3C758BAFD2AFD2A9D2ABD239
:02126E008E22CE
:100A140012125E7DA07F9012123D7D807F8E121295
:100A24003D12124CA2A1B3B0A250097B007A007906
:100A340047121186E4F5947593FFC2947F641211F2
:100A4400FED294A20592947B007A00792C120FFABC
:100A5400120AD520B00F20B00512001E80F8D20D66
:100A6400120CF5C20D300ADBE526B52ED6E524B509
:100A74002DD1AF541554EF700D7526FF7524FFC2A8
:100A84000A7554058041E5292553FF75F03B8425FB
:100A94002AF52AEF75F03B8485F029E52A75F00ADA
:100AA40084C454F0FFE52A75F00A84EF25F0F52696
:100AB400E52975F00A84C454F0FFE52975F00A8429
:100AC400EF25F0F524D20AD20D120CF5C20D020A5C
:010AD40047DA
:03000000020D8F5F
:0C0D8F00787FE4F6D8FD758154020DD683
:10095000C2D530F707B2D563F0FF05F030E70CB22F
:10096000D5F4048463F0FF05F080018430D502F4EF
:0209700004225F
:10097200BB010689828A83E0225002E722BBFE0283
:09098200E32289828A83E49322B6
:10098B00BB010689828A83F0225002F722BBFE014B
:02099B00F32245
:10099D00F8BB010DE58229F582E5833AF583E8F090
:1009AD00225006E92582C8F622BBFE05E92582C83C
:0209BD00F22224
:1009BF00BC000BBE0029EF8DF084FFADF022E4CC1C
:1009CF00F875F008EF2FFFEE33FEEC33FCEE9DECE5
:1009DF00984005FCEE9DFE0FD5F0E9E4CEFD22ED2B
:1009EF00F8F5F0EE8420D21CFEADF075F008EF2F75
:1009FF00FFED33FD4007985006D5F0F222C398FD66
:050A0F000FD5F0EA2202
:100D9B00020A14E493A3F8E493A34003F68001F250
:100DAB0008DFF48029E493A3F85407240CC8C33359
:100DBB00C4540F4420C8834004F456800146F6DF28
:100DCB00E4800B01020408102040809010DCE47ECC
:100DDB00019360BCA3FF543F30E509541FFEE4931D
:100DEB00A360010ECF54C025E060A840B8E493A3E4
:100DFB00FAE493A3F8E493A3C8C582C8CAC583CA0F
:100E0B00F0A3C8C582C8CAC583CADFE9DEE780BEC6
:0111230000CB
:00000001FF
